:10000E00323032322D30372D3132202D20313233F5
:05001E00343536370007
:1029D8007BFF7A00790E7D2D123E1EEA494B601F5F
:1029E8007BFF7A00790E7D2D123E1EE92402F9E460
:1029F8003AFA900257EBF0A3EAF0A3E9F08004E476
:102A0800FEFF22900257E0FBA3E0FAA3E0F9900052
:102A1800011210C3FF3395E0FEC3EF9430EE6480DB
:102A280094804016D3EF9439EE64809480500B90D4
:102A380000011210C324D0FF802E9000011210C391
:102A4800FF3395E0FEC3EF9461EE648094804016F6
:102A5800D3EF9466EE64809480500B9000011210BE
:102A6800C324A9FF80027F00EF7D00FC1210AAFF9B
:102A78003395E0FEC3EF9430EE64809480401ED31B
:102A8800EF9439EE648094805013900257E0FBA3D2
:102A9800E0FAA3E0F91210AA24D0FF80339002577D
:102AA800E0FBA3E0FAA3E0F91210AAFF3395E0FED9
:102AB800C3EF9461EE648094804013D3EF9466EE84
:102AC8006480948050081210AA24A9FF80027F0015
:102AD800EFC454F04CFC900257E0FBA3E0FAA3E0EB
:102AE800F99000021210C3FF3395E0FEC3EF943053
:102AF800EE648094804016D3EF9439EE648094801D
:102B0800500B9000021210C324D0FF803990025756
:102B1800E0FBA3E0FAA3E0F99000021210C3FF3330
:102B280095E0FEC3EF9461EE648094804016D3EF85
:102B38009466EE64809480500B9000021210C324B7
:102B4800A9FF80027F00EF75F010A4FFE5F04CFEAE
:102B5800EF4DFF900257E0FBA3E0FAA3E0F99000E5
:102B6800031210C3FD3395E0FCC3ED9430EC648090
:102B780094804016D3ED9439EC64809480500B9087
:102B880000031210C324D0FD8039900257E0FBA344
:102B9800E0FAA3E0F99000031210C3FD3395E0FCBE
:102BA800C3ED9461EC648094804016D3ED9466EC98
:102BB80064809480500B9000031210C324A9FD80F8
:062BC800027D00EF4DFF4D
:012BCE0022E4
:1026D400E47880F6124667C286E4F5A775E101F551
:1026E400E275E34043C910900255F0A3F0900256FE
:1026F400E004F07006900255E004F0900255E0709A
:1027040004A3E0640E70E643B28FE4F5A91245E534
:10271400E4FF12458543EF04E4900255F0A3F090E2
:102724000255E0FEA3E0FFC39402EE940050157D31
:1027340001124404900256E004F070E3900255E064
:1027440004F080DBE4F520C213C211C217C216C222
:10275400157880F608F67827F618F6782CF69002A5
:1027640055F0A3F0900255E0FEA3E0FFC3EE940100
:10277400501C74002FF58274003EF583E4F090023F
:1027840056E004F070DE900255E004F080D6E49048
:102794000255F0A3F0900255E0FEA3E0FFC394407D
:1027A400EE9400501C74002FF58274013EF583E40E
:1027B400F0900256E004F070DC900255E004F080E2
:1027C400D4E4F5A7E5EF54027010E5EF5408D39470
:1027D40000748094804003D38001C392037D08E495
:1027E400FF12453DE4782BF67824F69001F4E0FBE3
:1027F400A3E0FAA3E0F97824E6FF75F010A4F582CB
:1028040085F0831210C3FE782B26F6EE600578243B
:102814000680D8D3EF94007480948040359001F4FE
:10282400E0FBA3E0FAA3E0F990000D1213B9121033
:10283400AAFF74551210F01210AA64556002D21542
:1028440074AA1210F01210AA64AA6002D215EF1230
:1028540010F0E5EF5402D394007480948040047F18
:10286400018002E4FF122ED1900254EFF090025442
:10287400E05401703CC21274FF782EF608F608F694
:1028840008F67E007F107D007B007A0079341214F4
:102894004090026D74FFF0A3741EF0A374DFF0A3E4
:1028A400E4F0A37410F07B007A007934123FDF80E7
:1028B40002D2121229D87832A60608A6079002542A
:1028C400E0540260030229A0A3F0A3F0900256E0B2
:1028D400C4F8540FC868FF900255E0C454F048FE91
:1028E4009001F4E0FBA3E0FAA3E0F98F828E831257
:1028F40010C37003022997E92FF9EA3EFA90000405
:102904001210C320E27CE4900253F0900253E0FDE5
:10291400C3781F96506C900256E0C4F8540FC868F0
:10292400FF900255E0C454F048FE9001F4E0FBA38C
:10293400E0FAA3E0F98F828E831210C3FF7E00C0F9
:1029440006C0077C00900256E0C4F8540FC868FF24
:10295400900255E0C454F048FEE92FF9EA3EFA909B
:10296400000D1213B9782BE68DF0A429F9EA35F09D
:10297400FA7D00D007D006121440900253E004F010
:102984008089900256E004F07006900255E004F04D
:102994000228D07F011242D1C2148007E4FF124200
:1029A400D1D214E4900255F0A3F0900255E0FEA3B6
:1029B400E0FFC39402EE940050197A007B967D03E5
:1029C400123C8E900256E004F070DF900255E00451
:0329D400F080D7B9
:0129D70022DD
:05468A00782CE6FF2280
:03002300022D6249
:102D6200C0E0C0F0C083C082C0D075D000C000C037
:102D720001C002C003C004C005C006C00730997478
:102D8200C2997827067927E77881667030F6782726
:012D9200F64A
:102D930090023D740AF090023DE0D3940074809455
:102DA300804015000000000000000000000000004B
:082DB300000000E014F080DED6
:042DBB00C286803715
:102DBF0090023D7414F090023DE0D394007480941F
:102DCF00804015000000000000000000000000001F
:082DDF00000000E014F080DEAA
:102DE7007827E62400F582E43401F583E0F599209D
:102DF7009803022EB6209A08201305C298022EB215
:102E0700C29A7826E6062400F582E43400F583E5C5
:102E170099F0C298E6FF7E0064017013900000E00D
:102E2700FD7004F6022EB6ED54072402782DF6EF56
:102E370064024E700E782DE664097007900001E079
:102E47002403F67826E6FFFD7C00B40007ECB40106
:102E570003F6805BEFC3782D964054ED24FFFDEC1D
:102E670034FFFC7B017A00790012385E7826E6246D
:102E7700FFF582E434FFF583E06F60047600802F6E
:102E870090023D7414F090023DE0D3940074809456
:102E97008040150000000000000000000000000056
:082EA700000000E014F080DEE1
:102EAF0012002678267600D007D006D005D004D0A1
:102EBF0003D002D001D000D0D0D082D083D0F0D0B8
:022ECF00E032EF
:1037A600900001E075F010A4FF9001F4E0FBA3E0A7
:1037B600FAA3E02FF9EA35F0FA90000D1213B9904A
:1037C6000240782CE6FF18E68FF0A4FFE02FF58282
:0F37D600E435F0F5831210C3FF7B017A02793ED0
:1037E50090024DEFF0A3EBF0A3EAF0A3E9F090020D
:1037F5004EE0FBA3E0FAA3E0F9EA494B6022900210
:103805004EA3A31210AAFF90024DE0FD7C001246C4
:103815005890024EE0FBA3E0FAA3E0F9EF1210F096
:103825009002517414F0900251E0D3940074809486
:1038350080401500000000000000000000000000AE
:08384500000000E014F080DE39
:10384D0090024DE0F5997F011243CF3099FDC29959
:01385D002248
:103E98009001007478F07826E624FFF582E434FF78
:093EA800F583E0900101F07F02B6
:103EB10090FFFF12140FEFF090FFFF12140F850D0A
:0B3EC10083850E82A3E07881F6D28694
:103ECC00850D83850E827414F0850D83850E82E03A
:103EDC00D394007480948040150000000000000012
:0E3EEC00000000000000000000E014F080DB89
:0C3EFA00900100E0F59990000202140F06
:1040F000C9EFC9E964017028EDC39B403F781FE612
:10410000FFEB2FFFE433FEEDC39FEE6480F8748075
:10411000985029D213C3ED9B782CF678287601228B
:10412000CFE9CFEF6402701ACFEBCFCEEDCEEE6FBA
:10413000700AD213782CF67828760222C213E4781B
:0341400028F6223C
:103B760090024DECF0A3EDF0C9EFC9BAFF19BBFFF7
:103B86001690024DE06A7003A3E06B7068D213785A
:103B96002CF67828E9F622E964017035C390024EC6
:103BA600E09B90024DE09A4026781FE62BFFE43A10
:103BB600FEE0FCA3E0FDC39FEC9E5013D213CFEBB7
:103BC600CFCEEDCEC3EE9F782CF6782876012280F4
:103BD60024CFE9CFEF64027022CEEACECFEBCF90AE
:103BE600024DE06E7003A3E06F700AD213782CF6D4
:0C3BF6007828760222C213E47828F62218
:10002600900000E0FE54F890023FF0EE1213E90053
:100036007209007F0A009210009B1100AC1200C3E7
:100046001900D91A00FE2001042801B4290311332E
:1000560003523703923903AC4103B74903C2500434
:10006600166102DB70040E9800000446900001E061
:10007600FD782FE6FB7F018027900001E0FCA3E0DE
:10008600FD782EE6FA08E6FB7F01802BD21378284E
:100096007603020446900001E0FD7831E6FB7F021C
:1000A6001240F0020446900001E0FCA3E0FD783027
:1000B600E6FA08E6FB7F02123B7602044690000150
:1000C600E0FD782FE6FB7F011240F02013030204C7
:1000D60046801A900001E0FCA3E0FD782EE6FA08BF
:1000E600E6FB7F01123B76201303020446900100D3
:1000F6007478F07F0102044375EF10020446C2AC27
:10010600E490023EF0D2867B017A02793E7F7F122E
:1001160037E57B017A02793E7F181237E57B017A53
:1001260002793E7F051237E57824E61237DE782E0F
:10013600E61237DE782FE61237DE7830E61237DE43
:100146007831E61237DE7832E61237DE7833E61299
:1001560037DEE4900240F0900240E0FFC394107452
:10016600809480501074342FF8E61237DE900240E7
:10017600E004F080E290023EE0FF7B007A00790026
:030186001237E548
:1001890090024C740AF090024CE0D394007480946D
:100199008040150000000000000000000000000081
:0801A900000000E014F080DE0C
:1001B1000202C6900001E0FFC378249640030202C8
:1001C100CDEF75F010A4FF9001F4E0FBA3E0FAA3DA
:1001D100E02FF9EA35F0FA900249EBF0A3EAF0A337
:1001E100E9F0C2ACE490023EF0D2867B017A02795A
:1001F1003E7F7F1237E57B017A02793E7F0D123710
:10020100E5900249E0FBA3E0FAA3E0F91210AA127B
:1002110037DE900249E0FBA3E0FAA3E0F990000188
:100221001237DB900249E0FBA3E0FAA3E0F990006A
:10023100021237DB900249E0FBA3E0FAA3E0F99058
:1002410000031237DB900249E0FBA3E0FAA3E0F9D7
:100251009000041237DBE4900240F0900240E0FF8E
:10026100C39408748094805026900249E0FBA3E077
:10027100FAA3E02405F9E43AFA7E00E92FF9EE3A0F
:10028100FA1210AA1237DE900240E004F080CC90FE
:0D029100023EE0FF7B007A0079001237E5A5
:10029E0090024C740AF090024CE0D3940074809457
:1002AE00804015000000000000000000000000006B
:0802BE00000000E014F080DEF6
:1002C600C286D2AC0204469001007478F0E4A3F032
:1002D6007F02020443124680780F12133790010002
:1002E600747CF0780FE6A3F008E6A3F008E6A3F026
:1002F60008E6A3F07C007D057B017A0179001238BF
:100306005E900105EFF07F06020443900001E0FFD6
:100316007E006401700FA3E0FDA3E0782ECDF60801
:10032600EDF602040EEF64024E700A900002E078C9
:100336002EF602040E900001E06403700CA3E0FFA9
:10034600A3E07830CFF608EFF602040EE490024000
:10035600F0900240E0FFC394107480948050279080
:100366000001E0FEEFC39E501D900240E02402F51E
:1003760082E43400F583E0FE74342FF8EEF6900242
:1003860040E004F080CBE47843F6807C7A007B3250
:100396007D01782CE6FF123C8E900001E0FDE4FF23
:1003A60012453D020446900001E024FF9202020439
:1003B60046900001E024FF9201020446782CE66094
:1003C600089002427402F0800E90024220160574D4
:1003D60003F080037401F09001007479F0900242FA
:1003E600E0900101F07C007D027B017A0179001228
:1003F600385E900102EFF07F03123EB1900242E0B8
:100406006401703CD2178002D211788076F1803078
:100416007A007B327D017F00123C8E900100747958
:10042600F0900001E0900101F07C007D027B017AF2
:1004360001790012385E900102EFF07F03123EB19F
:1004460090023FE064A0600302070E781FE6640195
:10045600700AFA7B327D017F01123C8E900000E02B
:1004660064A160030205A9A3E0C3782496400302B1
:10047600059E9001F4E0FBA3E0FAA3E0F9900001E9
:10048600E0FF75F010A4F58285F0831210C3900288
:1004960042F0EF75F010A4FFE92FF9EA35F0FA9073
:1004A60000041210C330E23C900001E0FF1200038A
:1004B600900242EFF0900100747FF0A3EFF0240267
:1004C600FDE433FC7B017A01790012385E9002422A
:1004D600E0FE2402F582E43401F583EFF0EE240316
:1004E600FF02070B900001E0FF120003C2ACE4908C
:1004F600023EF0D286900242E0D394067480948045
:1005060040377B017A02793E7F7F1237E5900242BF
:10051600E01237DEE4900240F0900242E0FF9002E3
:1005260040E0C39F500B1237A6900240E004F080D3
:10053600E8900242E004F08026900242E02478121D
:1005460037DEE4900240F0900242E0FF900240E085
:10055600C39F500B1237A6900240E004F080E8904B
:0D056600023EE0FF7B007A0079001237E5CD
:1005730090024C740AF090024CE0D394007480947F
:100583008040150000000000000000000000000093
:08059300000000E014F080DE1E
:10059B000206FD9001007478F07F0102070B9000BA
:1005AB0000E064A2600302070E7824E6FFA3E0FEDE
:1005BB00C39F4003020703A3E0FDC39F4003020751
:1005CB0003EE9D4003020703900001E0900240F010
:1005DB00E4900247F0A3F0900002E0FE900240E0AE
:1005EB00FFD39E50341200039001F4E0FBA3E0FA1A
:1005FB00A3E0F9900240E075F010A4F58285F0833A
:10060B001210C3FF900248E02FF0900247E0340035
:10061B00F0900240E004F080BEC2ACE490023EF0E9
:10062B00D2867B017A02793E7F7F1237E5900247B3
:10063B00E0FEA3E0FFC39480EE94005002800F9085
:10064B000247E044801237DE900247A3E0FF1237E7
:10065B00DF900001E0900240F0900002E0FF90027A
:10066B0040E0D39F5056E4A3F09001F4E0FBA3E0ED
:10067B00FAA3E0F9900240E0FF75F010A4F5828533
:10068B00F0831210C3FE900241E0C39E5026EF751B
:10069B00F010A4FF9001F4A3A3E02FF9EA35F0FAD0
:1006AB0090000D1213B99002411237C8900241E02D
:1006BB0004F080B5900240E004F0809D90023EE093
:0A06CB00FF7B007A0079001237E58A
:1006D50090024C740AF090024CE0D394007480941C
:1006E5008040150000000000000000000000000030
:0806F500000000E014F080DEBB
:1006FD00C286D2AC800B9001007478F07F01123E5F
:10070D00B190023FE064587057FA7B327D01782C2E
:10071D00E6FF123C8E9002507401F0A37401F0A319
:10072D007401F07B017A007901124236900242EF9A
:10073D00F0E0FE2478900100F0EE2401FDE433FC9E
:10074D007B017A01790012385E900242E0FE2401AD
:10075D00F582E43401F583EFF0EE2402FF123EB191
:10076D0090023FE0FF64806008EF64886003020937
:10077D00807828E66401700EFA7B327D01782CE6D4
:10078D00FF123C8E8021E4900240F0900240E0FF89
:10079D00C3781F9650117A007B327D01123C8E90EA
:1007AD000240E004F080E4900000E0540790024223
:1007BD00F06407701290024104F0900001E0900285
:1007CD0042F09000028008E4900241F0900001E0B8
:1007DD00900243F0900242E014F0A3E0FFC37824AE
:1007ED009640030209809001F4E0FBA3E0FAA3E038
:1007FD00F975F010EFA4F58285F0831210C3FF9008
:10080D000242E0D39F4002EFF07828E66401700DBC
:10081D00782CE6900246F0900245F0800BE49002B1
:10082D0045F0781FE614A3F0900245E0782CF69081
:10083D000246E0FF782CE6D39F400302096EE49058
:10084D000240F0900242E0FF900240E0C39F40035F
:10085D00020960900243E075F010A4FF9001F4E0EE
:10086D00FBA3E0FAA3E02FF9EA35F0FA90000412A9
:10087D0010C330E2030209579000011210C364380F
:10088D007054900242E0D39404748094809002409E
:10089D00E0FF4011A3E02F2402F582E43400F5833C
:1008AD00E0FD0209377826E6C39FFFE49400FE744D
:1008BD00FE2FF58274FF3EF583E0FD900243E07557
:1008CD00F010A4FF9001F4E0FBA3E0FAA3E02FF9F0
:1008DD00EA35F0FA80549001F4E0FBA3E0FAA3E0CE
:1008ED00F9900243E075F010A4F58285F0831210A3
:1008FD00C3FF7826E6C39FFFE49400FE900240E01C
:10090D007C002FFFEC3EFEA3E02FFFEC3EFE74FFBC
:10091D002FF58274FF3EF583E0FD900243E075F004
:10092D0010A4FFE92FF9EA35F0FA90000D1213B972
:10093D00782CE6FF18E68FF0A4FF900240E02FF52B
:10094D0082E435F0F583ED121102900240E004F0DF
:10095D00020850900243E0FF12449A782C060208D8
:10096D003C900245E0782CF690023FE064887003DD
:10097D00123E9890023FE064A86003020B21782894
:10098D00E66401700EFA7B327D01782CE6FF123C95
:10099D008E8021E4900240F0900240E0FFC3781F6A
:1009AD009650117A007B327D01123C8E900240E010
:1009BD0004F080E4900001E030E718547FFEA3E0DE
:1009CD00FDEDFF900247EEF0A3EFF09002417403AE
:1009DD00F08013900001E0FF900247E4F0A3EFF0E8
:1009ED009002417402F0900241E0FF2400F582E490
:1009FD003400F583E0FE74012FF582E43400F583B5
:100A0D00E0900244F0CFEECF900243EFF09002441D
:100A1D00E0FF900243E0FED39F4003020B1EEEC3A6
:100A2D007824964003020B159001F4E0FBA3E0FA45
:100A3D00A3E0F975F010EEA4F58285F0831210C3D2
:100A4D00900242F07828E66401700D782CE6900251
:100A5D0046F0900245F0800BE4900245F0781FE6D9
:100A6D0014A3F0900245E0782CF6900246E0FF7852
:100A7D002CE6D39F4003020B03E4900240F090025A
:100A8D0042E0FF900240E0C39F505D900243E0754D
:100A9D00F010A4FF9001F4E0FBA3E0FAA3E02FF91E
:100AAD00EA35F0FA9000041210C320E233900240B0
:100ABD00E0FFA3E02F2402F582E43400F583E0FD8E
:100ACD0090000D1213B9782CE6FF18E68FF0A4FFF5
:100ADD00900240E02FF582E435F0F583ED1211021E
:100AED00900240E004F08096900243E0FF12449A99
:100AFD00782C06020A77900245E0782CF690024297
:100B0D00E0FF900241E02FF0900243E004F0020A72
:040B1D001A123E98D2
:010B210022B1
:10F000007880E664F1600302FA157819F608F6785C
:04F0100081E66039FC
:10F01400900253740AF0900253E0D39400748094E5
:10F024008040150000000000000000000000000007
:08F03400000000E014F080DE92
:10F03C00781A06E6187001067819B627C608B610B5
:10F04C00C2C2AFE47815F618F620984BE47819F69E
:10F05C0008F620983EC3781AE6948818E694135064
:01F06C003271
:10F06D00900253740AF0900253E0D394007480948C
:10F07D0080401500000000000000000000000000AE
:08F08D00000000E014F080DE39
:10F09500781A06E61870C20680BFB29780B2781457
:10F0A500A699C298E6FF641A6008EF640A60030235
:10F0B500F218E47819F608F620983EC3781AE69413
:07F0C5008818E69413503295
:10F0CC00900253740AF0900253E0D394007480942D
:10F0DC00804015000000000000000000000000004F
:08F0EC00000000E014F080DEDA
:10F0F400781A06E61870C20680BF20980302F055FD
:10F104007815A699C298E47819F608F620983EC3B3
:0BF11400781AE6948818E69413503235
:10F11F00900253740AF0900253E0D39400748094D9
:10F12F0080401500000000000000000000000000FB
:08F13F00000000E014F080DE86
:10F14700781A06E61870C20680BF20980302F055A9
:10F157007815A699C298E47819F608F620983EC360
:0BF16700781AE6948818E694135032E2
:10F17200900253740AF0900253E0D3940074809486
:10F1820080401500000000000000000000000000A8
:08F19200000000E014F080DE33
:10F19A00781A06E61870C20680BF20980302F05556
:10F1AA007815A699C29818E6641A600302FA06D27C
:03F1BA0086C29971
:10F1BD009002537414F0900253E0D3940074809431
:10F1CD00804015000000000000000000000000005D
:08F1DD00000000E014F080DEE8
:06F1E5007599783099FDD8
:10F1EB00900253740AF0900253E0D394007480940D
:10F1FB00804015000000000000000000000000002F
:08F20B00000000E014F080DEB9
:10F21300C28602FA067814E6FF7E00645060030299
:10F22300F3367819F608F620983EC3781AE69488E0
:06F2330018E694135032AE
:10F23900900253740AF0900253E0D39400748094BE
:10F2490080401500000000000000000000000000E0
:08F25900000000E014F080DE6B
:10F26100781A06E61870C20680BF20980302F0558E
:0AF271007815A699C298D286C299BA
:10F27B009002537414F0900253E0D3940074809472
:10F28B00804015000000000000000000000000009E
:08F29B00000000E014F080DE29
:08F2A3007599793099FDC299BB
:10F2AB009002537414F0900253E0D3940074809442
:10F2BB00804015000000000000000000000000006E
:08F2CB00000000E014F080DEF9
:08F2D3007599013099FDC29903
:10F2DB009002537414F0900253E0D3940074809412
:10F2EB00804015000000000000000000000000003E
:08F2FB00000000E014F080DEC9
:06F30300E4F5993099FDCC
:10F30900900253740AF0900253E0D39400748094ED
:10F31900804015000000000000000000000000000F
:08F32900000000E014F080DE9A
:10F33100C28602FA06EF64014E600302F3CED28662
:02F34100C2996F
:10F343009002537414F0900253E0D39400748094A9
:10F3530080401500000000000000000000000000D5
:08F36300000000E014F080DE60
:08F36B007599783099FDC299F3
:10F373009002537414F0900253E0D3940074809479
:10F3830080401500000000000000000000000000A5
:08F39300000000E014F080DE30
:06F39B00E4F5993099FD34
:10F3A100900253740AF0900253E0D3940074809455
:10F3B1008040150000000000000000000000000077
:08F3C100000000E014F080DE02
:10F3C900C28602FA067814E66402600302F506783A
:10F3D90019F608F620983EC3781AE6948818E69438
:03F3E9001350328C
:10F3EC00900253740AF0900253E0D394007480940A
:10F3FC00804015000000000000000000000000002C
:08F40C00000000E014F080DEB6
:10F41400781A06E61870C20680BF20980302F055D9
:10F424007815A699C298E408F618E6FF13B39297E4
:10F43400EF25E0FECC74F0CCCD7400CDC3E49DEE9A
:10F444009C502AE67F0025E0FEC39460501FE4F53B
:10F45400A7758F03781BEEF608EFF675B7A57880CD
:10F46400E6F5B78F828E83E4F0F58F800478167604
:05F47400FFD286C299E1
:10F479009002537414F0900253E0D3940074809472
:10F48900804015000000000000000000000000009E
:08F49900000000E014F080DE29
:08F4A1007599783099FDC299BC
:10F4A9009002537414F0900253E0D3940074809442
:10F4B900804015000000000000000000000000006E
:08F4C900000000E014F080DEF9
:08F4D1007816E6F5993099FD6B
:10F4D900900253740AF0900253E0D394007480941C
:10F4E900804015000000000000000000000000003E
:08F4F900000000E014F080DEC9
:10F50100C28602FA067814E66403600302F6E07824
:10F5110019F608F620983EC3781AE6948818E694FE
:03F5210013503252
:10F52400900253740AF0900253E0D39400748094D0
:10F5340080401500000000000000000000000000F2
:08F54400000000E014F080DE7D
:10F54C00781A06E61870C20680BF20980302F055A0
:10F55C007815A699C298E47819F608F620983EC357
:0BF56C00781AE6948818E694135032D9
:10F57700900253740AF0900253E0D394007480947D
:10F58700804015000000000000000000000000009F
:08F59700000000E014F080DE2A
:10F59F00781A06E61870C20680BF20980302F0554D
:10F5AF007817A699C2987815E6FF139297EF25E082
:10F5BF00FECC74F0CCCD7400CDC3E49DEE9C400323
:10F5CF0002F055E625E0FCC39460400302F055E4D9
:10F5DF00F5A7758F017817E675F020A42400FFE5D5
:10F5EF00F03C781BF608EFF6E47818F67818E6C3C7
:10F5FF009420748094805047E408F608F6209816FB
:10F60F00C3781AE6948818E69413500A000806E6A1
:10F61F001870EA0680E720980302F05575B7A578B1
:10F62F0080E6F5B7781B0806E618CEE6CE70010621
:10F63F0014F5828E83E599F0C29878180680ADE4B0
:06F64F00F58FD286C2997E
:10F655009002537414F0900253E0D3940074809494
:10F6650080401500000000000000000000000000C0
:08F67500000000E014F080DE4B
:08F67D007599783099FDC299DE
:10F685009002537414F0900253E0D3940074809464
:10F695008040150000000000000000000000000090
:08F6A500000000E014F080DE1B
:06F6AD00E4F5993099FD1F
:10F6B300900253740AF0900253E0D3940074809440
:10F6C3008040150000000000000000000000000062
:08F6D300000000E014F080DEED
:10F6DB00C28602FA067814E6FD7C0064046003021D
:10F6EB00F80B7819F608F620983EC3781AE694883A
:06F6FB0018E694135032E2
:10F70100900253740AF0900253E0D39400748094F1
:10F711008040150000000000000000000000000013
:08F72100000000E014F080DE9E
:10F72900781A06E61870C20680BF20980302F055C1
:10F739007815A699C298E625E0781DF608E4F678CA
:10F7490016F67819F608F6781D0806E618CEE6CEFC
:10F7590070010614F5828E83E493781626F6781ADA
:10F7690006E618700106781AE6700418E664027055
:05F77900D6D286C29902
:10F77E009002537414F0900253E0D394007480946A
:10F78E008040150000000000000000000000000096
:08F79E00000000E014F080DE21
:08F7A6007599783099FDC299B4
:10F7AE009002537414F0900253E0D394007480943A
:10F7BE008040150000000000000000000000000066
:08F7CE00000000E014F080DEF1
:08F7D6007816E6F5993099FD63
:10F7DE00900253740AF0900253E0D3940074809414
:10F7EE008040150000000000000000000000000036
:08F7FE00000000E014F080DEC1
:10F80600C28602FA06ED64054C600302F9FC78191B
:10F81600F608F620983EC3781AE6948818E69413FC
:02F8260050325E
:10F82800900253740AF0900253E0D39400748094C9
:10F8380080401500000000000000000000000000EB
:08F84800000000E014F080DE76
:10F85000781A06E61870C20680BF20980302F05599
:10F860007815A699C298E47819F608F620983EC350
:0BF87000781AE6948818E694135032D2
:10F87B00900253740AF0900253E0D3940074809476
:10F88B008040150000000000000000000000000098
:08F89B00000000E014F080DE23
:10F8A300781A06E61870C20680BF20980302F05546
:0AF8B3007817A699C298D286C29970
:10F8BD009002537414F0900253E0D394007480942A
:10F8CD008040150000000000000000000000000056
:08F8DD00000000E014F080DEE1
:08F8E50075997F3099FDC2996D
:10F8ED009002537414F0900253E0D39400748094FA
:10F8FD008040150000000000000000000000000026
:08F90D00000000E014F080DEB0
:10F915007599203099FD7815E625E0FC7817E67590
:10F92500F020A42400FFE5F03C781DF608EFF6E48E
:10F935007816F67818F67818E6C3942074809480C3
:04F945005057C299BC
:10F949009002537414F0900253E0D394007480949D
:10F9590080401500000000000000000000000000C9
:08F96900000000E014F080DE54
:10F97100781DE6FE08E6F5828E83E493F5993099C9
:10F98100FD781D0806E618CEE6CE70010614F58254
:0FF991008E83E493781626F6781806809DC29927
:10F9A0009002537414F0900253E0D3940074809446
:10F9B0008040150000000000000000000000000072
:08F9C000000000E014F080DEFD
:08F9C8007816E6F5993099FD6F
:10F9D000900253740AF0900253E0D3940074809420
:10F9E0008040150000000000000000000000000042
:08F9F000000000E014F080DECD
:10F9F800C286800A7814E66406700375EF107814DE
:0DFA0800E66407600302F0557880F6D2AF87
:01FA150022CE
:103F06007F001243CF20120B7A007B327D017F00A7
:103F1600123C8E30150B7A007B1E7D017F00123C11
:103F26008E3011173016147A007B327D01782CE61C
:103F3600FF123C8EC211123605D21220140C301616
:103F460009788076F1123605D21430170B30160830
:103F5600C21712466712F000201612124676E47B4C
:0E3F66002C7A01F9F8C312131A5002D2162257
:1044C60075EF027F64EFD394007480948040031FDD
:1044D60080F31226D412468A124601E4FFFE1243E6
:0944E60056123F0612300F80F857
:10314C00005EBCE2613FDD83C29C7E20A3FD1F417B
:10315C009DC3217FFCA2401E5F01E3BD3E6082DC6B
:10316C00237D9FC1421CFEA0E1BF5D0380DE3C625B
:10317C00BEE0025CDF81633D7C22C09E1D43A1FF4B
:10318C004618FAA427799BC584DA3866E5BB59073B
:10319C00DB856739BAE406581947A5FB7826C49A2B
:1031AC00653BD987045AB8E6A7F91B45C6987A241B
:1031BC00F8A6441A99C7257B3A6486D85B05E7B90B
:1031CC008CD2306EEDB3510F4E10F2AC2F7193CDFB
:1031DC00114FADF3702ECC92D38D6F31B2EC0E50EB
:1031EC00AFF1134DCE90722C6D33D18F0C52B0EEDB
:1031FC00326C8ED0530DEFB1F0AE4C1291CF2D73CB
:10320C00CA947628ABF517490856B4EA6937D58BBA
:10321C005709EBB536688AD495CB2977F4AA4816AA
:10322C00E9B7550B88D6346A2B7597C94A14F6A89A
:10323C00742AC896154BA9F7B6E80A54D7896B358A
:0A324C000000000000002B96B9DD21
:03461A00014D0A45
:10460100900253121368FFFFFFFF900253E0FCA3D7
:08461100E0FDA3E0FEA3E0FFC1
:01461900227E
:10385E0090FFFE12140FECF0A3EDF090FFFD12148A
:0F386E000FEBF0A3EAF0A3E9F090FFFC12140FA8
:10387D00850D83850E82A3A3E4F0850D83850E82CD
:10388D00F0A3F0900007121433E0FEA3E0FF850DC6
:10389D0083850E82E0FCA3E0FDC39FEE6480F8EC0F
:1038AD00648098504C900004121433E0FBA3E0FAAE
:1038BD00A3E0F98D828C831210C3FF850D83850ED5
:1038CD0082A3A3E06FFF900003121433EFF090007A
:1038DD0003121433E090314C93850D83850E82A332
:1038ED00A3F0850D83850E82E475F0011211AF8072
:0B38FD0092850D83850E82A3A3E0FFDF
:0639080090000902140FFB
:0E465800CEEDCEEE6F7813F6E690314C93FF68
:014666002231
:10453D00EF7020F5A77598D0E589540F4420F589C3
:10454D00438E08CFEDCFEF90324B93F58DD28ED2B7
:05455D00ACC2BCD2AFAE
:014562002236
:10404700785012134F00000000785412134F0000ED
:10405700000078447664E47814F67814E6C3940292
:1040670074809480502EE6FF25E025E02445F8E48F
:10407700F6EF25E025E02446F8E4F6EF25E025E015
:104087002447F8E4F6EF25E025E02448F8E4F6783D
:04409700140680C6C5
:01409B002202
:1045E500D2AFD2A9C2BBE589540F4401F589758EB6
:0C45F50002758CECE4F58AD28C02404781
:0636E20090FFFF12140F1F
:1036E800850D83850E82E4F0850D83850E82E0FFCB
:1036F800C394027480948040030237A0EF25E0252C
:10370800E02448F8E6FF7C00D3940074809480405D
:1037180069E025E025E02446F8E6705EEF30E00D2C
:10372800D394017480948040047D0080087D0185D5
:103738000D83850E82E0FF123F74850D83850E820E
:10374800E0FF25E025E02448F8E6640170057D01E6
:10375800123F74850D83850E82E0FF25E025E02465
:1037680048F816E66014EF25E025E02447F8E6FE61
:10377800EF25E025E02446F8EEF6850D83850E82D8
:10378800E025E025E02446F8E6600116850D8385EE
:083798000E82E004F00236F09D
:0637A00090000102140F6D
:03000B00023D169D
:103D1600C0E0C0F0C083C082C0D0E8C0E0E9C0E027
:103D2600EAC0E0EBC0E0ECC0E0EDC0E0EEC0E0EFE2
:103D3600C0E0758CEC785012132BEF2401FFE43EA3
:103D4600FEE43DFDE43CFC7850121337784416E659
:103D5600701B785412132BEF2401FFE43EFEE43D62
:103D6600FDE43CFC7854121337784476641236E24C
:103D7600124563D0E0FFD0E0FED0E0FDD0E0FCD0FD
:103D8600E0FBD0E0FAD0E0F9D0E0F8D0D0D082D095
:063D960083D0F0D0E03202
:1044040090FFFF12140FEDF090FFFF12140FEFF066
:10441400850D83850E82E0FFC394027480948050DE
:104424000DA3E0FEEF25E025E02445F8EEF690002C
:044434000202140F5D
:103C8E0090FFFE12140FEAF0A3EBF090FFFF121458
:103C9E000FEDF090FFFF12140FEFF0850D83850EE0
:103CAE0082E0FFC39402748094805056EF25E02585
:103CBE00E02448F8E6704BE0FB25E025E02446F8CA
:103CCE00E6703FA3E025E004FF850D83850E82E0BC
:103CDE00FA25E025E02448F8EFF6850D83850E825F
:103CEE00A3A3E0FEA3E0FF7C007D0A121179EA2572
:103CFE00E025E02447F8EFF6EB25E025E02446F832
:083D0E00E4F690000402140F1A
:103F740090FFFF12140FEDF090FFFF12140FEFF0FB
:103F8400850D83850E82E0FFFD7C00C3940274805E
:103F94009480501EEF25E025E02445F8E66013A345
:103FA400E070047F0180027F00850D83850E82A36B
:103FB400EFF0ED4C700E850D83850E82A3E024FF97
:103FC40092978011850D83850E82E064017006A3AB
:0B3FD400E024FF92A090000202140FF6
:09467600C2AF785012132BD2AF31
:01467F002218
:09468000C2AF785412132BD2AF23
:01468900220E
:1043CF0090FFFF12140FEFF0850D83850E82E070C2
:1043DF0005784EF608F6301816784DE675F064A499
:1043EF00FFC3784FE69F18E695F05003E4F5D3909E
:0543FF00000102140F93
:10458500D218E4784EF608F6EF784D6003F680020F
:10459500760AE4F5D975D2FF75D940F5D375EF06DE
:0145A50022F3
:0F466700C218E4784EF608F6784D76FFF5D922A2
:10456300784F06E618700106301816784DE675F098
:1045730064A4FFC3784FE69F18E695F05003E4F573
:02458300D32241
:08435600900253EEF0A3EFF01A
:10435E00E4A3F0A3F0900253E0FEA3E0FFC39002AB
:10436E0056E09F900255E09E501C7FE87E03123D62
:10437E009C7F011243CF900256E004F070D790025A
:06438E0055E004F080CFB1
:014394002206
:083D9C00900257EEF0A3EFF0D6
:103DA400D394FAEE94005024900257A3E0FFEFD38B
:103DB4009400748094804061007E03EED394007478
:103DC4008094804004001E80F21F80E2900257E03D
:103DD400FFA3E0A3CFF0A3EFF0D390025AE094FA4C
:103DE400900259E0940040177FFA7E00123D9C90A7
:103DF400025AE02406F0900259E034FFF080DAD34E
:103E0400900258E09400900257E09400400B900216
:093E140059E0FEA3E0FF123D9C01
:013E1D002282
:103A4C009002637401F0A37402F0A3745DF07B0127
:063A5C007A02795B7D0295
:0E3A620090025FEBF0A3EAF0A3E9F0A3EDF011
:103A70007F011243CF900263E0FBA3E0FAA3E0F9D9
:103A80001211DB2400FFE5F03460FE90025FE0F9E4
:103A9000A3E0FAA3E0900266C9F0A3EAF0A3E9F07C
:103AA000E4FD900262E0FCEDC39C5022EF2DF58214
:103AB000E43EF583E493FC900266E0FBA3E0FAA306
:103AC000E0F98D82758300EC1211020D80D4900212
:103AD00062E0FFA3E0FBA3E0FAA3E0F9E48FF002C9
:023AE0001206CC
:103526009002557412F0A37434F090025D7401F0A9
:10353600A37402F0A37457F07B017A0279557D02D9
:0E354600900259EBF0A3EAF0A3E9F0A3EDF038
:103554007880E664F16003023604124667C2AFE481
:10356400F5A7758F01A3E0FBA3E0FAA3E0F912111C
:10357400DB2400FFE5F034607814F608EFF69002DF
:1035840059E0FBA3E0FAA3E0F97818C6EBC608C635
:10359400EAC608C6E9C6E47816F690025CE0FF784D
:1035A40016E6C39F503C7818CBE6CB080806E6180D
:1035B400CAE6CA70010614F91210AA7817F675B78C
:1035C400A57880E6F5B77817E6FF78140806E618BC
:1035D400CCE6CC70010614F5828C83EFF0781606E5
:1035E40080B8E4F58F90025CE0FFA3E0FBA3E0FA6F
:1035F400A3E0F9E48FF0121206D2AFE4FF1245857E
:0136040022A3
:1041E6007880E664F17048C2AF124667E4F5A775B9
:1041F6008F037815766008F67814F67814E6C3947B
:104206000874809480501F75B7A57880E6F5B77856
:1042160015E6FE08E6F5828E83E4F026F6187402AB
:0F42260036F6180680D5E4F58FD2AFFF12458526
:014235002266
:103605001241E6E4900257F0A3F07B0190025D04BD
:10361500F0A37402F0A37457F01B7A00792E7D167F
:10362500123546123526E4900254F0900254E0C358
:10363500781F9640030236DAE4900253F09001F4C5
:10364500E0FBA3E0FAA3E0F9900253E0FF75F01068
:10365500A4F58285F0831210C36071EF75F010A494
:10366500FF9001F4A3A3E02FF9EA35F0FA90000DDD
:103675001213B9900254E0FF782BE68FF0A429F9D4
:10368500EA35F0FAEBC0E0EAC0E0E9C0E09001F409
:10369500E0FBA3E0FAA3E0F9900253E075F010A473
:1036A500F58285F0831210C3FD90025D7401F0A3CD
:1036B5007402F0A37457F0D0E0F9D0E0FAD0E0FB43
:1036C500123546900253E004F0023642900254E06F
:0C36D50004F0023630123526E47880F64E
:0136E10022C6
:052ED100900257EFF034
:102ED600E490025DF0A3F090025AF07B0190026349
:102EE60004F0A37402F0A3745DF01B7A00792E7DC2
:102EF60016123A62123A4C90025BE0B4120CA3E04E
:102F0600B4340790025AE04401F0E4900259F0907C
:102F16000259E0C3781F964003022FF3E49002584B
:102F2600F09001F4E0FBA3E0FAA3E0F9900258E088
:102F3600FF75F010A4F58285F0831210C3700302AA
:102F46002FEA900257E0606AEF75F010A4FF900137
:102F5600F4A3A3E02FF9EA35F0FA90000D1213B9A5
:102F6600900259E0FF782BE68FF0A429F9EA35F0B4
:102F7600FAEBC0E0EAC0E0E9C0E09001F4E0FBA3B0
:102F8600E0FAA3E0F9900258E075F010A4F5828506
:102F9600F0831210C3FD9002637401F0A37402F073
:102FA600A3745DF0D0E0F9D0E0FAD0E0FB123A620B
:102FB60080299001F4E0FBA3E0FAA3E0F99002581F
:102FC600E075F010A4F58285F0831210C3FF90021D
:102FD6005EE02FF090025DE03400F0900258E004CD
:102FE600F0022F27900259E004F0022F15123A4CF6
:102FF60090025BE0B4120CA3E0B4340790025AE0EE
:083006004402F090025AE0FFC1
:01300E00229F
:101EDF004D50444300013400000043484E30000091
:101EEF000000010142013400000043484E31000060
:101EFF000000010143013400000043484E3200004E
:101F0F000000010144013400000043484E3300003B
:101F1F000000010145013400000043484E34000029
:101F2F000000010146013400000043484E35000017
:101F3F000000010147013400000043484E36000005
:101F4F000000010148013400000043484E370000F3
:101F5F000000010149013400000043484E380000E1
:101F6F00000001014A013400000043484E390000CF
:101F7F00000001014B013400000043484E31300096
:101F8F00000001014C013400000043484E31310084
:101F9F00000001014D013400000043484E31320072
:101FAF00000001014E013400000043484E31330060
:101FBF00000001014F013400000043484E3134004E
:101FCF000000010150013400000043484E3135003C
:101FDF000000010151013400000043484E3136002A
:101FEF000000010152013400000043484E31370018
:101FFF000000010153013400000043484E31380006
:10200F000000010154013400000043484E313900F3
:10201F000000010155013400000043484E323000EA
:10202F000000010156013400000043484E323100D8
:10203F000000010157013400000043484E323200C6
:10204F000000010158013400000043484E323300B4
:10205F000000010159013400000043484E323400A2
:10206F00000001015A013400000043484E32350090
:10207F00000001015B013400000043484E3236007E
:10208F00000001015C013400000043484E3237006C
:10209F00000001015D013400000043484E3238005A
:1020AF00000001015E013400000043484E32390048
:1020BF00000001015F013400000043484E3330003F
:1020CF000000010160013400000043484E3331002D
:1020DF00000001016104060000014930000000000A
:1020EF0000000101620406000001493100000000F8
:1020FF0000000101660406000001493200000000E3
:10210F00000001016A0406000001493300000000CD
:10211F00000001016E0406000001493400000000B8
:10212F0000000101720406000001493500000000A3
:10213F00000001017604060000014936000000008E
:10214F00000001017A040600000149370000000079
:10215F00000001017E040600000149380000000064
:10216F00000001018204060000014939000000004F
:10217F000000010186040600000149313000000013
:10218F00000001018A0406000001493131000000FE
:10219F00000001018E0406000001493132000000E9
:1021AF0000000101920406000001493133000000D4
:1021BF0000000101960406000001493134000000BF
:1021CF00000001019A0406000001493135000000AA
:1021DF00000001019E040600000149313600000095
:1021EF0000000101A2040600000149313700000080
:1021FF0000000101A604060000014931380000006B
:10220F0000000101AA040600000149313900000055
:10221F0000000101AE040600000149323000000049
:10222F0000000101B2040600000149323100000034
:10223F0000000101B604060000014932320000001F
:10224F0000000101BA04060000014932330000000A
:10225F0000000101BE0406000001493234000000F5
:10226F0000000101C20406000001493235000000E0
:10227F0000000101C60406000001493236000000CB
:10228F0000000101CA0406000001493237000000B6
:10229F0000000101CE0406000001493238000000A1
:1022AF0000000101D204060000014932390000008C
:1022BF0000000101D6040600000149333000000080
:1022CF0000000101DA04060000014933310000006B
:1022DF0000000101DE04080000015430000000007E
:1022EF0000000101E2040800000154310000000069
:1022FF0000000101E6040800000154320000000054
:10230F0000000101EA04080000015433000000003E
:10231F0000000101EE0132000000506F776572007E
:10232F0000000101F201320000004572726F72006D
:10233F0000000101F3000000000000000000000099
:05234F00000000000089
:0E461D00011F014301F4FF1EE44201400000B2
:1042D100EF6022E4FFEFC394207480948050107447
:1042E100422FF582E43401F5837401F00F80E690EA
:1042F10001F27401F0E4F5A775A45D75A5FF75A63B
:1043010087D28112463012344512428690023B74A4
:0243110001F0B9
:014313002287
:10449A0090FFFF12140FEFF0850D83850E82E0FF67
:1044AA007E00C39420748094804005EF64447006B3
:0C44BA0090023B7401F090000102140F0E
:0800030090024DEFF07F002296
:1042360090024DEBF0A3EAF0A3E9F090024DE0FB0B
:10424600A3E0FAA3E0F91210AAFF900250E0FBA344
:10425600E0FAA3E0F9EF1210F090024DE0FBA3E0C4
:10426600FAA3E0F99000011210C3FF900250E0FBA0
:10427600A3E0FAA3E0F9900001EF1211027F0222F7
:10300F0012149390023BE06065E4F09001F2E064EB
:10301F0001703B900253F0900253E0FFC394207471
:10302F00809480504974422FF582E43401F583E097
:10303F00540164019002537006E0FF7D018004E0AB
:10304F00FFE4FD1239B0900253E004F080C9E49020
:10305F000253F0900253E0FFC39420748094805089
:10306F000DE4FD1239B0900253E004F080E51246F2
:10307F0076ECC0E0EDC0E0EEC0E0EFC0E0900140C4
:10308F00E0FEA3E0FFCBEFCBCAEECAD0E0FFD0E06B
:10309F00FED0E0FDD0E0FCC3EF9BFFEE9AFEED9477
:1030AF0000FDEC9400FCE47B64FAF9F8C312131AE8
:1030BF00400302314B124676900140EEF0A3EFF041
:1030CF007B017A017942122BCFE4900253F09002E8
:1030DF0053E0C3942074809480502DE0FE1313139B
:1030EF00541FFFEE54072402FD123256900253E094
:1030FF0025E025E02462F582E43401F583121343C1
:10310F00900253E004F080C6E4900253F090025313
:10311F00E0FFC39404748094805021E4FD12325672
:10312F00900253E025E025E024E2F582E43401F536
:0C313F0083121343900253E004F080D18F
:01314B002261
:10463000E4F5A7C280C282D291D294D292D293D210
:0646400095D296D2A122E2
:10431400E4F5A7EF14B40700503790432C75F0036D
:10432400A4C58325F0C58373024341024344024379
:104334004702434A02434D024350024353C291226F
:10434400C29422C29222C29322C29522C29622C24F
:02435400A122A4
:10464600E4F5A7D291D294D292D293D295D296D2B1
:02465600A1229F
:10443800E4F5A7FEEEC39408748094805020EF54EE
:10444800019400748094804003D38001C39282EF6A
:10445800C313FFD280D280D280C2800E80D6C2829F
:014468002231
:10446900E4F5A7FEEEC39408748094805020EF54BD
:10447900809400748094804003D38001C39282EFBA
:1044890025E0FFD280D280D280C2800E80D6C2823F
:014499002200
:1044EF00E4F5A7FFC282FEEEC39408748094805057
:1044FF0015EF25E0FFA281E4334FFFD280D280D2A7
:06450F0080C2800E80E175
:014515002283
:102354000000000000000040404040400000606079
:102364006060600000707070707000007878787839
:102374007800007C7C7C7C7C00007E7E7E7E7E00FF
:10238400007F7F7F7F7F00000609090600000000B0
:102394000000000000000000000000000000000039
:1023A4000000000000000000000000000000000029
:1023B4000000000000000000000000000000000019
:1023C4000000000000000000000000000000000009
:1023D40000000000000000000000000000000000F9
:1023E40000000000000000000000000000000000E9
:1023F40000000000000000000000000000000000D9
:1024040000000000000000000000000000000000C8
:1024140000000000000000000000000000000000B8
:1024240000000000000000000000000000000000A8
:102434000000000000000000005F00000000040332
:102444000004030000147F147F140000242A7F2A50
:1024540012000063130864630000304E512E5000D4
:102464000000040300000000001C224100000000E2
:1024740041221C0000002A1C7F1C2A000008083E80
:1024840008080000004030000000000808080808A0
:1024940000000060600000000060100804030000F9
:1024A4003E5149453E000000427F40000000426129
:1024B4005149460000224149493600001814127F50
:1024C400100000274545453900003C4A4949300081
:1024D4000001710905030000364949493600000628
:1024E4004949291E00000036360000000000563617
:1024F40000000000081422410000001414141414F5
:1025040000000041221408000002015109060000E5
:102514003E415D555E00007C1211127C00007F4933
:1025240049493600003E414141220000417F41417A
:102534003E00007F4949414100007F090909090023
:10254400003E4141517200007F0808087F000000EE
:10255400417F41000000204040403F00007F0814BC
:10256400224100007F4040404000007F0204027F7F
:1025740000007F0408107F00003E4141413E0000FE
:102584007F0909090600003E4151215E00007F09D0
:1025940019294600002649494932000001017F01FA
:1025A4000100003F4040403F00001F2040201F002A
:1025B400007F2018207F00006314081463000003C8
:1025C40004780403000061514945430000007F4141
:1025D40041000000030408106000000041417F0036
:1025E400000004020102040000404040404000009A
:1025F40000070B000000003844443C4000007F50BA
:1026040048483000003844444420000030484850D2
:102614007F000038545454080000087E090200006A
:1026240000081454543C00007F080404780000009F
:10263400487A400000002040443D0000007F1028FC
:102644004400000000417F40000000780408047842
:1026540000007C0804047800003844444438000036
:102664007C142424180000182424147C0000007C0A
:10267400080404000048545454200000043F44203B
:102684000000003C4040207C00001C2040201C0036
:10269400003C4030403C0000442810284400000422
:1026A4004830080400004464544C440000000836D8
:1026B40041000000000077000000000041360800DF
:1026C4000000000408100800007F7F7F7F7F000067
:1045C600D2A27F071243147F7F1244691246467FA8
:0F45D600071243147F80124469124646C2A22284
:0B3AE20090026AEBF0A3EAF0A3E9F009
:103AED007F07124314E4900270F090026DF0900283
:103AFD006DE0FFC3940874809480506A90026AE070
:103B0D00FBA3E0FAA3E0F98F827583001210C39036
:103B1D00026FF07003A304F0900270E06005E49072
:103B2D00026FF0E490026EF090026EE0FFC3940518
:103B3D00748094805028A3E075F007A42454F58276
:103B4D00E5F03423F583E5822FF582E43583F583A3
:103B5D00E493FF12446990026EE004F080CA900273
:093B6D006DE004F0808802464678
:10390E00486F6C6420256300486F6C64202020256E
:10391E0063003E3E3E4F4E3C3C3C002D2D4F4646F6
:10392E002D2D004F56455254454D50004F56455281
:10393E004355525200505752204F4E00505752206E
:10394E004F464600434825303262643A464C540096
:10395E00434825303262643A257300454E0044498F
:10396E0053004925303262643A25332E31664100C8
:10397E00542562643A25342E316608004D53434275
:10398E003A256400323032332D31312D3238202D2C
:10399E002034363835353830002D2D2D2D2D2D2D4A
:0239AE002D00EA
:04462B004102BE008A
:1043950020A4047F0180027F00EF25E025E0FF20B7
:1043A500A3047E0180027E00EE75F008A44FFF2075
:1043B500A5047E0180027E00EE25E04FFF20A604C5
:0A43C5007E0180027E00EF4EFF2211
:10149300124676E47B32FAF9F8D312131A40099014
:1014A30002BEE07003021A5B9002BEE07033124585
:1014B300C69002BE7401F0A312136800000000E49A
:1014C3009002C3F0A3F0A3F0A3121368000000007E
:1014D3009002CA12136800000000E49002CEF0A349
:1014E300F01246769002BFE0F8A3E0F9A3E0FAA376
:1014F300E0FBC3EF9BFFEE9AFEED99FDEC98FCE455
:101503007B0AFAF9F8D312131A4003021A5B124644
:10151300769002BF121343E4900265F0900264F0E8
:10152300900263F0900262F0124395900261EFF033
:101533009002CEE0704E900261E0FF30E30D900226
:10154300C3E020E3069002637401F0EF30E20D90F4
:1015530002C3E020E2069002627401F0900261E0AF
:1015630020E10D9002C3E030E1069002647401F0C3
:10157300900261E020E00D9002C3E030E0069002AB
:10158300657401F0900261E0FF7E0070049002CE6A
:10159300F0EF4E60091246769002CA1213431246C8
:1015A30076A804A905AA06AB079002CAE0FCA3E04B
:1015B300FDA3E0FEA3E02470FFEE3417FEE43DFD3F
:1015C300E43CFCD312131A4005E49002CFF09002DE
:1015D300CFE0640270199002C5E02442F9E43401BB
:1015E300FA9002667401F0A3EAF0A3E9F0800E908A
:1015F30002667401F0A37401F0A374F2F090026127
:10160300E020E1030216D1900266E0FBA3E0FAA317
:10161300E0F91210AA540160030216D19002C3E04C
:1016230020E1091246769002C612134312467690C1
:1016330002C6E0F8A3E0F9A3E0FAA3E0FBC3EF9B43
:10164300FFEE9AFEED99FDEC98FCE47B0AFAF9F8BB
:1016530012127A900269EFF07E00C39405748094AD
:1016630080406B9002CE7401F090026D74FFF0A382
:101673007439F0A3740EF0EF24FBFFEE34FFC313B1
:10168300EF13A3F07B017A027954121AC17B017A1A
:10169300027954123AE2900269E0C394147480947C
:1016A300804028900266E0FBA3E0FAA3E0F974010E
:1016B3001210F09002CFE0640290023B700504F038
:1016C3000217A47401F0E49001F3F00217A490024E
:1016D30061E020E0030217AD900266E0FBA3E0FAAD
:1016E300A3E0F91210AA5401640160030217AD903C
:1016F30002C3E020E0091246769002C61213431299
:1017030046769002C6E0F8A3E0F9A3E0FAA3E0FB73
:10171300C3EF9BFFEE9AFEED99FDEC98FCE47B0A88
:10172300FAF9F812127A900269EFF07E00C3940579
:101733007480948040749002CE7401F090026D74B2
:10174300FFF0A37439F0A37416F0EF24FBFFEE341B
:10175300FFC313EF13FFC374079FA3F07B017A0248
:101763007954121AC17B017A027954123AE2900237
:1017730069E0C39414748094804026900266E0FB71
:10178300A3E0FAA3E0F9E41210F09002CFE06402C0
:1017930090023B700404F080087401F0E49001F3BC
:1017A300F0900261E09002C3F022900261E09002A7
:1017B300C3F0900262E060139002CFE02401FFE4E3
:1017C30033FE7C007D07121124EDF0900263E0608C
:1017D300139002CFE02406FFE433FE7C007D071262
:1017E3001124EDF09002CFE0B407004003021A5B2E
:1017F3009017FAF828287302180F02185502187266
:101803000218FB0219620219C90219F49001F3E0EC
:10181300701D9001F2E0D39400748094807BFF40AC
:10182300077A397920021A587A397929021A589095
:1018330001F3E030E0097BFF7A397931021A5890DD
:1018430001F3E020E103021A5B7BFF7A39793A0264
:101853001A589001F2E0D39400748094807BFF4087
:10186300077A397943021A587A39794A021A589011
:1018730002C5E0FF2442F582E43401F583E030E25F
:101883001290026D74FFF0A37439F0A37452F0A3A5
:10189300EF803990026D74FFF0A37439F0A3745E86
:1018A300F09002C5E0900270F02442F582E4340126
:1018B300F583E07BFF30E0067A39796980047A3971
:1018C300796C900271EBF0A3EAF0A3E9F07B017A63
:1018D300027954121AC17B017A027954123AE290C6
:1018E3000264E060089002C5E004541FF0900265B2
:1018F300E07003021A5B805D90026D74FFF0A374C5
:1019030039F0A37470F09002C5E0900270F025E006
:1019130025E02462F582E43401F583E0FCA3E0FDD5
:10192300A3E0FEA3E0FF9002711213437B017A024E
:101933007954121AC17B017A027954123AE2900265
:1019430064E060089002C5E004541FF0900265E073
:101953007003021A5B9002C5E0241F541FF022900B
:10196300026D74FFF0A37439F0A3747EF09002C487
:10197300E0900270F025E025E024E2F582E43401F2
:10198300F583E0FCA3E0FDA3E0FEA3E0FF9002717A
:101993001213437B017A027954121AC17B017A0232
:1019A3007954123AE2900264E060089002C4E004C1
:1019B3005403F0900265E07003021A5B9002C4E0E6
:1019C30024035403F02290026D74FFF0A37439F0E2
:1019D300A3748AF0782EE6FF08E6A3CFF0A3EFF016
:1019E3007B017A027954121AC17B017A02795480FD
:1019F300647BFF7A3979927D2D123E1EEA494B7B37
:101A0300FF604E7A3979927D2D123E1EE92402F948
:101A1300E43AFA90025EEBF0A3EAF0A3E9F0900255
:101A2300547423F090025EE0F9A3E0FAA3E090027D
:101A33006DC9F0A3EAF0A3E9F0A3E4F0A37407F0FF
:101A43007B017A027955123FDF7B017A0279548058
:081A5300047A3979A7123AE286
:011A5B002268
:10344500E4F5A7C290FE7F0CFD7B017A0279A612F6
:103455001440E4900257F0900257E0FFC3942074A3
:103465008094805042EF75F003A4FFAEF07C007DA0
:103475000812117974A62FF58274023EF583C08374
:10348500C082E0FF900257E075F003A45407FEF8F0
:103495007401088002C333D8FC4FD082D083F090EA
:1034A5000257E004F080B0E4900257F0900257E034
:1034B500FFC3940C748094805014749A2FF582E4A1
:1034C5003402F583E4F0900257E004F080DEE490E6
:1034D5000257F0900257E0FFC39406748094805021
:1034E5003F7B087D0A124195900257E0FF25E024B5
:1034F500A6F582E43402F583E0F4FBE4FD12419580
:10350500900257E0FF25E024A7F582E43402F58315
:10351500E0F4FB7D01124195900257E004F080B381
:013525002283
:10419500900259EDF0A3EBF0900258EFF0C39403B1
:1041A5007480948050047F0180027F021243149032
:1041B5000258E0C39403748094804004E02405F021
:1041C500900258E0540725E04440FF1244699002EC
:1041D50059E0FF12446990025AE0FF124469024611
:0141E5004693
:0A409C0090025BEDF090025AEFF085
:1040A600C394037480948050047F0180027F0212BF
:1040B600431490025AE0C39403748094804004E051
:1040C60024FDF090025AE0540725E04441FF1244D3
:1040D6006990025BE0FF1244691244EF90025CEFC4
:0940E600F012464690025CE0FF76
:0140EF0022AE
:0239B000AC0762
:1039B200EC75F003A4FBAAF0EAC4F854F0C8EBC417
:1039C200540F48900255F0AE02EB7803CEC313CEEB
:1039D20013D8F9900254F0EC75F003A45407FFEDEC
:1039E2006401701EE0249AF582E43402F583C083F8
:1039F200C082E0FEA8077401088002C333D8FC4EDF
:103A02008020900254E0249AF582E43402F583C0C7
:103A120083C082E0FEA8077401088002C333D8FC89
:103A2200F45ED082D083F0900255E0FF900254E021
:103A3200FE540170047D1480027D15749A2EF58265
:0A3A4200E43402F583E0FB02419535
:0B2BCF00900254EBF0A3EAF0A3E9F041
:102BDA00E4A3F0900257E0C3940C74809480502AC6
:102BEA00E0FEC313FFEE540170047D1280027D13D0
:102BFA0012409C900257E024B2F582E43402F58335
:102C0A00EFF0900257E004F080C9E4900257F09088
:102C1A000257E0C39420748094804003022CBAE0E7
:102C2A00FD75F003A42401FFE435F0FEEF7803CE2E
:102C3A00C313CE13D8F9900258F0ED75F003A4042B
:102C4A005407A3F0900258E024B2F582E43402F566
:102C5A0083E0FD7C00900259E0FF7E007401A80722
:102C6A00088005C333CE33CED8F9FFEE5CFEEF5DA4
:102C7A004E9002546018E0FBA3E0FAA3E0F9A3E047
:102C8A00FFE92FF9E43AFA1210AA44028016E0FB8F
:102C9A00A3E0FAA3E0F9A3E0FFE92FF9E43AFA1274
:102CAA0010AA54FD1210F0900257E004F0022C19F9
:102CBA00E4900257F0900257E0C394207480948005
:102CCA004003022D61E0FD75F003A42402FFE43500
:102CDA00F0FEEF7803CEC313CE13D8F9900258F062
:102CEA00ED75F003A424025407A3F0900258E024DF
:102CFA00B2F582E43402F583E0FD7C00900259E0EB
:102D0A00FF7E007401A807088005C333CE33CED8EE
:102D1A00F9FFEE5CFEEF5D4E9002547018E0FBA3E3
:102D2A00E0FAA3E0F9A3E0FFE92FF9E43AFA121076
:102D3A00AA44048016E0FBA3E0FAA3E0F9A3E0FFAB
:102D4A00E92FF9E43AFA1210AA54FB1210F0900291
:072D5A0057E004F0022CBF5A
:012D6100224F
:0841430090025CEDF0A3EBF02B
:10414B00EF2403FF12431490025CE0C454F0FFA36E
:10415B00E0540F4FFF124469E4900262F090026149
:10416B00E0FFA3E0C39F501F1244EF90025EE0FB01
:10417B00A3E475F0011211C5A9F0FAEF1210F0903B
:0A418B000262E004F080D60246460E
:1045A600900258EDF0A3EBF0EF2403FF12431490B2
:1045B6000258E0C454F0FFA3E0540F4FFF024469D1
:03468F000246469A
:0346920002446976
:10428600E4900257F0900257E0FFC39404748094C0
:10429600805037E4FB7D071245A6900257E0FFE405
:1042A600FB7D0D1245A67FFF1246927FFF124692B6
:1042B600E4FF124692E4FF1246927F1512469212CE
:0A42C600468F900257E004F080BB21
:0142D00022CB
:06325600900254EDF0FBB4
:10325C0090025E7401F0A37402F0A37455F0A37491
:10326C0002F0FD124143900255E0C4F854F0C868D6
:10327C00FCA3E0C4540F48FDE4120DC5E4FBFA793D
:10328C00207840120C1AE4FBFA79807845120D2351
:10329C00900257121343900254E0900257704CE086
:1032AC00FCA3E0FDA3E0FEA3E0FF7BCD7ACC794C40
:1032BC007843120C1A900257121343E4FFFE7D2040
:1032CC007C41900257E0F8A3E0F9A3E0FAA3E0FBFD
:1032DC00120C1AE4FBFAF9783F120B29123355E45D
:1032EC00FBFA79207841120D238015E0FCA3E0FD58
:1032FC00A3E0FEA3E0FFE4FBFA79207841120C1A5C
:10330C00900257121343E4FFFE7DC87C4290025793
:10331C00E0F8A3E0F9A3E0FAA3E0FB120C1AE4FB3B
:10332C00FAF9783F120B29123355E4FBFA79C87875
:10333C0042120D23900257121343900257E0FCA344
:08334C00E0FDA3E0FEA3E0FF99
:013354002256
:100B2200020E33E86480F8E933E83360110460F0C0
:100B3200ED33EC337009E8FCE9FDEAFEEBFF220439
:100B420060DED3EB9FEA9EE99DE8C2E78CF0C2F734
:100B520095F0400CE8CCF8E9CDF9EACEFAEBCFFB00
:100B6200120DFE85D0F05804700320D5B3E804704E
:100B7200075002B2D5020E3D92D5EC0460F7E4CCE8
:100B8200C0E0C398F8603B94186008400DD0E0FBC9
:100B9200020E15E4FBFAC9FC8028E830E406E4C939
:100BA200FBE4CAFCE830E305E4C9CACBFCE854071D
:100BB2006010F8C3E913F9EA13FAEB13FBEC13FC28
:100BC200D8F130F52FC3E49CFCEF9BFFEE9AFEEDCB
:100BD20099FDD0E0FBEF4E4D4C701222DB03020E6A
:100BE2003AEC2CFCEF33FFEE33FEED33FDED30E754
:100BF200EB020E15EF2BFFEE3AFEED39FDD0E0FBD6
:100C020050130BBB0003020E3DED13FDEE13FEEF7E
:080C120013FFEC13FC020E15A8
:100C1A00EC4D6011E8497017ED33EC3304600DE4D4
:100C2A00FCFFFEFD22E933E8330470F8020E3312AA
:100C3A000DFE58046009E4CC2481500628500902AC
:100C4A000E3D284003020E3AC0E0EB4A7044B980D8
:100C5A0006D0E0FB020E29EF4E701CBD8008EBFFA8
:100C6A00EAFEE9FD80EBE98DF0A4FEE5F0020D0352
:100C7A00E9CDF9EAFEEBFFEF89F0A4FCE5F0CE89B5
:100C8A00F0A42EFFE435F0CD89F0A42DFEE435F072
:100C9A008067EF4E7005BD80D780C3EF8BF0A4ACA0
:100CAA00F0EE8BF0A42CFCE435F0F8EF8AF0A42CDB
:100CBA00E5F038FCE433CB8DF0A42CFCE5F03BF8EE
:100CCA00EE8AF0A42CFCE5F038F8E433CF89F0A4DE
:100CDA002CFCE5F038CF3400CE89F0A42FFFE5F0E4
:100CEA003EFEE433C98DF0A42EFEE5F039CD8AF03C
:100CFA00A42FFFE5F03EFEE43DFD33D0E0FB5007B4
:100D0A000BBB000F020E3DEC2CFCEF33FFEE33FE63
:060D1A00ED33FD020E1591
:100D2000020E3DEC5D046005E859047003020E33C9
:100D3000120DFE580460F6EC4860F2EC7004FDFE03
:100D4000FF22C860DB2481C85009C39860025006A6
:100D5000020E3A9850CAF582E9294B4A7005AB82D7
:100D6000020E2975F0007C1A7880C3EF9BEE9AED95
:100D700099400DC3EF9BFFEE9AFEED99FDE842F01E
:100D8000DC23ACF0D0E0FFD0E0FED0E0FDAB822071
:100D9000E7101BEB60BAEC2CFCEF33FFEE33FEEDFB
:100DA00033FD020E15E803F830E705C0F075F000DA
:100DB000EF2FFFEE33FEED33FD40B830E7C280AADF
:100DC00075F020800E75F010800575F0087D007EAE
:100DD000007F003392D530D50312130CEC33401052
:100DE000EF33FFEE33FEED33FDEC33FCD5F0ED22B7
:0E0DF000E5F0247EA2D513CC92E7CDCEFF22F3
:101A5C00E508246DF582E43402F583E00508229054
:101A6C00026A300F0390026DE475F00112139902B3
:101A7C0010AA2008E97F2ED2088018EF540F24906A
:101A8C00D43440D4FF300C0BEF24BFB41A005003F5
:101A9C002461FFE50960021509050CE50C700205CF
:101AAC000B300F0E90026AE475F001121399EF02DD
:101ABC0010F00245167403D20F8003E4C20FF50830
:101ACC0090026A1213B0E4F509F50BF50CE5096008
:101ADC00077F20121A9F80F5750AFFC209C208C23F
:101AEC000AC20BC20DC20EC210121A6BFF700D305F
:101AFC000F057F00121AB0AF0CAE0B22B4255FC2DB
:101B0C00D5C20C121A6BFF24D0B40A00501A75F00F
:101B1C000A780930D50508B6FF0106C6A426F620BA
:101B2C00D5047002D20B80D924CFB41A00EF500424
:101B3C00C2E5D20C021DA2D20980C6D20880C0D246
:101B4C000A80BCD2D580BAD20D80B47F20121A9FE5
:101B5C00200A077401B5090040F1121A5CFF121A31
:101B6C009F021AD9D210D20E8095121A5CFB121A4F
:101B7C005CFA121A5CF94A4B700679A07A1E7BFF4C
:101B8C00200A2EE509602A7E008E827583001210D1
:101B9C00C360060EEE650A70F0C2D5EBC0E0EAC079
:101BAC00E0E9C0E0EE121E03D0E0F9D0E0FAD0E09C
:101BBC00FB1210AAFF60AAEBC0E0EAC0E0E9C0E0AB
:101BCC00121A9FD0E02401F9D0E03400FAD0E0FBE7
:101BDC00E50A0460DCD50AD98087D20A80A2121DDE
:101BEC00E560F7E50A700104120EF8A90A600DE52C
:101BFC000A600914F50A121E8DEF60F3EA30E70251
:101C0C00F404C3995079EAF4250A0430E701E4049A
:101C1C00F50A800D121DE560C1EA050A250A120EAF
:101C2C00F8EA900299F030E701E4250A04D50A0499
:101C3C00200D0114121E03E4C0E0121E8D900299B7
:101C4C00E0601320E70714F0121A87802204F0D00A
:101C5C00E014C0E07F00121A87E50A6007121A7EB2
:101C6C00150A800B300D03121A7ED0E0021AD9D05F
:101C7C00E00480C4121DE5609EE50A04120EF89083
:101C8C000299EAF0E50A200D026001042404121EF8
:011C9C000344
:101C9D0074FF04C0E0121E8D121A87E50A200D0292
:101CAD006003121A7ED0E0B50AE87F45121A9190B2
:101CBD000299E07F2B30E7047F2DF404C0E0121A67
:101CCD009FD0E075F00A84C0F0121A88D0E0121A85
:101CDD0088021AD9791080027908C20EC2108008C4
:101CED00D2D5790A8004790AC2D5E50A047002F5C5
:101CFD000AE4FAFDFEFF121A5CFC7B0820091312A0
:101D0D001A5CFD7B1030080A121A5CFE121A5CFF79
:101D1D007B20EC3382D592D55013C3E43008069F57
:101D2D00FFE49EFEE42009039DFDE49CFCE4CBF85A
:101D3D00C209EC700CCFCECDCCE824F8F870F3804E
:101D4D0017C3EF33FFEE33FEED33FDEC33FCEB3316
:101D5D00FB994002FB0FD8E9EB300905F8D0E0C440
:101D6D0048B209C0E00AEC4D4E4F78207B0070C29E
:101D7D00EAB50A0040BCC0E0121E05D0F0D0E0204C
:101D8D000904C4C0E0C4B209C0F0121A88D0F0D55D
:101D9D00F0EB021AD91213E91B76531CE1581B47BD
:101DAD004C1B43421CE54F1CED441CED491B5C4391
:101DBD001CF3551C20461C80451BEA471EC0501BBA
:101DCD004B2D1B4F2E1B722B1B53231B70201EA93B
:101DDD002A1B0B4800001B6AE50AB4FF03750A06AF
:101DED00121A5CFC121A5CFD121A5CFE121A5CFFD0
:101DFD00900292020F35790AA2D5200B14300D09ED
:101E0D00B910020404B9080104A2D5200E02500134
:101E1D0004200A68920AB509005034C0E07F2030D2
:101E2D000B197F30A20A720E720D500F121E5CC27A
:101E3D000AC20EC20DC2107F30800F300D03E9C0F3
:101E4D00E0121A9F300D03D0E0F9D0E0B509CC3087
:101E5D000D177F30B9100C121A9F7F58300C077F69
:101E6D00788003B90803121A9F300A057F2D021AD4
:101E7D009F7F202010F87F2B200EF322920A80CF17
:101E8D007F00B40700500B2492F582E43402F583F1
:101E9D00E0FF22286E756C6C2900D209121A5C3095
:101EAD0009F8C209780930D50108F6021B0B2D502F
:101EBD00434958121A5C2403B405004001E4901EF6
:101ECD00BB93121A90743A121A90D20B7509040230
:021EDD001CE106
:1033550090025B12134374FFFFFEFDFC90025BE0DD
:10336500F8A3E0F9A3E0FAA3E0FBC312131A60384F
:103375007F807E967D187C4B90025BE0F8A3E0F998
:10338500A3E0FAA3E0FB120E486002501B7F807E8B
:10339500967D187CCB90025BE0F8A3E0F9A3E0FAF8
:1033A500A3E0FB120E48500F90025BE0FCA3E0FD8A
:1033B500A3E0FEA3E0FF2290025BE0FCA3E0FDA3F7
:1033C500E0FEA3E0FF120EC190025F1213439002CC
:1033D5005FE0FCA3E0FDA3E0FEA3E0FFEC120DC05F
:1033E500C8ECC8C9EDC9CAEECACBEFCB90025BE009
:1033F500FCA3E0FDA3E0FEA3E0FF120B25E4FBFA2E
:10340500F9F8120E486026402490025FE0FCA3E024
:10341500FDA3E0FEA3E0FFEF24FFFFEE34FFFEED8A
:1034250034FFFDEC34FFFC90025F12134390025F02
:10343500E0FCA3E0FDA3E0FEA3E0FFEC120DC0223B
:100DFE00E9D2E7C933E833F892D5EDD2E7CD33EC3B
:070E0E0033FC5002B2D522B3
:100E1500EC30E7100FBF000C0EBE00080DBD00043E
:100E25000BEB6014A2D5EB13FCED92E7FD2274FFEA
:100E3500FCFDFEFF22E480F8A2D574FF13FC7D8043
:030E4500E480EF57
:100E480074F8CC6480CCC86480C8F58204604FC351
:100E5800EB9FF5F0EA9E42F0E99D42F0E89C45F0F0
:100E6800603C501DE5825FFFE582D313CB5BCBF47A
:100E78002B5582FB50280ABA002409B900200880A3
:100E88001DE5825BFBE582D313CF5FCFF4C3132F3D
:100E98005582FF50090EBE00050DBD00010CC3EBC5
:100EA8009FF5F0EA9E42F0E99D42F0E89C45F0602B
:090EB80007CC4820E701B3EC224D
:100EC100EDD2E7CD33EC3392D524814006E4FFFE29
:100ED100FDFC22FCE4CFCECDCC24E0501174FF8088
:100EE100EDC3CC13CCCD13CDCE13CECF13CF047025
:070EF100F030D5DE02130C06
:100EF800F920E73624F950037907E4F42402FBE5E6
:100F080082158270021583DBF6E024FB501BE96032
:100F180014E4F0E582158270021583E004F0B40A47
:0D0F280008E4F0D9EE7401F00A22C2D522CF
:100F3500ED33EC3392D5FA602AB4FF33EDC2E77B8B
:100F4500FF60067A0F795AE4227A0F796320D50477
:100F55007A0F795E224E614E002B494E46002D498F
:100F65004E4600E47A08F0A3DAFC7B00740722C041
:100F750083C082ECC0E0EDC0E0EEC0E0EFC0E0EA87
:100F850075F010A4CAABF075F04DA42BFBE435F059
:100F9500FCEA2410FAEB34C5FBEC34D9FCEDC2E7CE
:100FA500FF75F056A4F42411C5F0F434C58FF0A4F0
:100FB5002AE5F03BE43CF020E71412106AD0E0FF8C
:100FC500D0E0FED0E0FDD0E0FC120D238014F40447
:100FD50012106AD0E0FFD0E0FED0E0FDD0E0FC12B8
:100FE5000C1AD082D083E0FAEDD2E7CD33EC33246E
:100FF50082FBE4C3CF33CFCE33CECD33CD33DBF35A
:101005007B0775F00A846004F0A31B0AE5F0F0A3E2
:101015008FF0740AA4FFACF08EF0740AA42CFEAC19
:10102500F050010C8DF0740AA42CFDE435F0F0A30A
:05103500DBDE74072260
:10103A003F8000004120000042C80000447A0000BE
:10104A00461C400047C35000497424004B18968040
:10105A004CBEBC205A0E1BCA6753C21C749DC5AE37
:10106A00FB60065407601C2323121098EB54386067
:10107A0009121084121093120C1AECF8EDF9EEFA18
:10108A00EFCB22EB12109380F1543803241C9010FA
:10109A003AFE93FC0EEE93FD0EEE930ECE93FF22D4
:03000000023C02BD
:0C3C0200787FE4F6D8FD758181023C4912
:1010AA00BB010689828A83E0225002E722BBFE0244
:0910BA00E32289828A83E4932277
:1010C300BB010CE58229F582E5833AF583E02250E2
:1010D30006E92582F8E622BBFE06E92582F8E2222C
:0D10E300E58229F582E5833AF583E4932246
:1010F000BB010689828A83F0225002F722BBFE01DF
:02110000F322D8
:10110200F8BB010DE58229F582E5833AF583E8F023
:10111200225006E92582C8F622BBFE05E92582C8CF
:02112200F222B7
:10112400BC000BBE0029EF8DF084FFADF022E4CCAF
:10113400F875F008EF2FFFEE33FEEC33FCEE9DEC78
:10114400984005FCEE9DFE0FD5F0E9E4CEFD22EDBE
:10115400F8F5F0EE8420D21CFEADF075F008EF2F08
:10116400FFED33FD4007985006D5F0F222C398FDF9
:051174000FD5F0EA2296
:10117900C2D5EC30E709B2D5E4C39DFDE49CFCEE91
:1011890030E715B2D5E4C39FFFE49EFE121124C3D4
:10119900E49DFDE49CFC800312112430D507C3E4CF
:0611A9009FFFE49EFE2200
:1011AF00C5F0F8A3E028F0C5F0F8E58215827002CB
:0611BF001583E038F02268
:1011C500A3F8E0C5F025F0F0E582158270021583DD
:0611D500E0C838F0E8223A
:1011DB00BB010A89828A83E0F5F0A3E022500687DF
:1011EB00F009E71922BBFE07E3F5F009E3192289A1
:0B11FB00828A83E493F5F074019322D4
:10120600BB010789828A830211AF500B09C5F027FB
:10121600F7C5F01937F722BBFE0D09F8E325F0F301
:10122600C5F019E338F322F889828A83740193257D
:08123600F0C5F0F8E493382242
:10123E0075F008758200EF2FFFEE33FECD33CDCC67
:10124E0033CCC58233C5829BED9AEC99E5829840EA
:10125E000CF582EE9BFEED9AFDEC99FC0FD5F0D6C7
:10126E00E4CEFBE4CDFAE4CCF9A88222B800C1B9F1
:10127E000059BA002DEC8BF084CFCECDFCE5F0CB2F
:10128E00F97818EF2FFFEE33FEED33FDEC33FCEB68
:10129E0033FB10D703994004EB99FB0FD8E5E4F923
:1012AE00FA227818EF2FFFEE33FEED33FDEC33FC10
:1012BE00C933C910D7059BE99A4007EC9BFCE99A04
:1012CE00F90FD8E0E4C9FAE4CCFB2275F010EF2F49
:1012DE00FFEE33FEED33FDCC33CCC833C810D70749
:1012EE009BEC9AE899400AED9BFDEC9AFCE899F884
:0E12FE000FD5F0DAE4CDFBE4CCFAE4C8F92217
:0E130C00C3E49FFFE49EFEE49DFDE49CFC22F2
:10131A00EB9FF5F0EA9E42F0E99D42F0E89C45F029
:01132A0022A0
:0C132B00E6FC08E6FD08E6FE08E6FF22EE
:0C133700ECF608EDF608EEF608EFF622E2
:0C134300ECF0A3EDF0A3EEF0A3EFF0221D
:10134F00D083D082E493F608740193F60874029365
:09135F00F608740393F67404739C
:10136800A8828583F0D083D08212137F12137F1254
:10137800137F12137FE473E493A3C583C5F0C58379
:10138800C8C582C8F0A3C583C5F0C583C8C582C8CF
:011398002232
:10139900F8E0FBA3A3E0F925F0F0E58215827002DD
:0713A9001583E0FA38F02281
:0913B000EBF0A3EAF0A3E9F0223E
:1013B900BB010DE58229F582E5833AF583021475AF
:1013C9005007E92582F802146CBBFE07E92582F86B
:1013D90002147EE58229F582E5833AF583021487B2
:1013E900D083D082F8E4937012740193700DA3A393
:1013F90093F8740193F5828883E4737402936860A7
:06140900EFA3A3A380DFA6
:10140F00E50E2582F582E50D3583F583B50D04854F
:10141F00820E2210AF0685820EF50D2285820EF503
:04142F000DD2AF2209
:0D143300E50E2582F582E50D3583F5832257
:10451600EFB40A07740D124521740A309811A89950
:10452600B8130CC2983098FDA899C298B811F63005
:0745360099FDC299F59922DD
:103FDF0090026AEBF0A3EAF0A3E9F0E4900272F02A
:103FEF00A3F090027074FFF5F01211C545F0603C1C
:103FFF0090026DE0FBA3E0FAA3E0F91210AAFF9084
:10400F00026AE0FBA3E0FAA3E0F9900272E475F014
:10401F00011211C585F082F583EF121102EF60C214
:10402F0090026EE475F0011211AF80B690026AE053
:08403F00FBA3E0FAA3E0F92263
:103E1E0090026AEBF0A3EAF0A3E9F0A3EBF0A3EAB9
:103E2E00F0A3E9F090026DE0FBA3E0FAA3E0F91233
:103E3E0010AA600C90026EE475F0011211AF80E4CE
:103E4E0090026DE0FBA3E0FAA3E0F91210AA6D70E8
:103E5E00012290026AE0FBA3E0FAA3E0F9EBC0E0D6
:103E6E00EAC0E0E9C0E0A3E0FBA374FFF5F0121195
:103E7E00C5FAD082D083D0E06B7009E5F065827010
:0A3E8E0003EA658370BAFBFAF9221B
:10144000EF4E6012EF60010EEDBB010B89828A83C3
:10145000F0A3DFFCDEFA2289F05007F709DFFCA9D0
:0C146000F022BBFEFCF309DFFCA9F02227
:103C0E000244C6E493A3F8E493A34003F68001F2C2
:103C1E0008DFF48029E493A3F85407240CC8C333B7
:103C2E00C4540F4420C8834004F456800146F6DF86
:103C3E00E4800B010204081020408090461AE47EB6
:103C4E00019360BCA3FF543F30E509541FFEE4937B
:103C5E00A360010ECF54C025E060A840B8E493A342
:103C6E00FAE493A3F8E493A3C8C582C8CAC583CA6D
:103C7E00F0A3C8C582C8CAC583CADFE9DEE780BE25
:01462F00008A
:09146C00E6FB08E6FA08E6F922A5
:09147500E0FBA3E0FAA3E0F92278
:09147E00E2FB08E2FA08E2F9229F
:0C148700E493FB740193FA740293F922C1
:00000001FF
